:1000000012C0189518951895189518951895189563
:100010005EC81895189518951895189518951895FF
:100020001895189518958FE58DBFC0E4EEE24E2E19
:1000300084E08EBFD4E0F4E05F2EEEEFF3E0A0E6C4
:10004000B0E088278D933197E9F78CE089B980E09B
:1000500080BD88E18AB954D966248FEF81BB8FEFC8
:1000600087BB80E084BBAA9AAB9A979883E088BB51
:10007000C09880E08FBD85E08EBD85E086B980ECBC
:1000800087B9379A7894EEE9F0E080E481D958E0B6
:10009000C895802D77D931965A95D1F704C015109F
:1000A0001F1F1F1F1015EEEBF0E088E471D958E018
:1000B000C895802D67D931965A95D1F704C015019E
:1000C0001F1F1F1F0115EEEDF0E080E561D958E01C
:1000D000C895802D57D931965A95D1F704C00C1286
:1000E000120C20202020EEEFF0E088E551D958E0F6
:1000F000C895802D47D931965A95D1F704C015205F
:10010000202020202015EEE1F1E080E641D958E0E2
:10011000C895802D37D931965A95D1F704C015204E
:100120001F1F1F1F2015EEE3F1E080E731D958E0D3
:10013000C895802D27D931965A95D1F704C015104E
:10014000101010101015EEE5F1E088E721D958E005
:10015000C895802D17D931965A95D1F704C015014D
:10016000010101010115AFD88CE012D9A398ABECC5
:10017000B0E09C9197FF04C09B9B0EC09F779C931F
:100180009B990AC089E19F93992735D99F919B99A3
:1001900003C090689C9301C0A6C18D9AE4E6F0E08C
:1001A00088EC90E00197959A16D9959814D9482F24
:1001B000492BC1F7E0E0F0E0A0E1B0E0E4DC0F3F64
:1001C00009F004C084E68093C80005C0E0E0F0E0D8
:1001D000A8ECB0E0D8DC8FE711E084D8E0E2FDE1E4
:1001E0006AD88FEB11E07ED8EAE3FDE164D8A398EA
:1001F000ABECB0E09C9197FF04C09B990EC09F7739
:100200009C939B9B0AC089E19F939927F4D89F9167
:100210009B9B03C090689C9301C0CCCFA8EAB0E040
:100220008C918F5F8C9380EC806C87B9E4D9A5E7C3
:10023000B0E08D939C93A5E7B0E08D919C91A9ECE3
:10024000B0E08D939C93A5E7B0E00D911C9142E046
:1002500050E00AD8A9ECB0E04D935C930091A8005F
:10026000053008F001C04BC08FE711E03BD8E4E552
:10027000FDE121D8A9ECB0E00D911C910A3050E0CD
:10028000150708F009C002E011D8A6E1B4E0E9ECD6
:10029000F0E0F3DB03D82AC0A9ECB0E00D911C918B
:1002A000093050E0150780E010F009F081E08F93ED
:1002B000A9ECB0E00D911C91043650E0150781E0E7
:1002C00008F080E09F918923882309F409C001E0A8
:1002D000EDD7A6E1B4E0E9ECF0E0CFDBDFD706C074
:1002E000A6E1B4E0E9ECF0E0C8DBD8D780E0809389
:1002F000A8008FEB11E0F6D7E8E5FDE1DCD78FE74A
:1003000017E0F0D7A9ECB0E00D911C914BE150E063
:10031000ABD7A4EAB0E04D935C9382E18093A9004F
:1003200082E18093AA0068D6A398ABECB0E09C91E0
:1003300097FF04C09B9B0EC09F779C939B990AC01C
:1003400089E19F93992757D89F919B9903C0906803
:100350009C9301C063CF8D9AE4E6F0E088EC90E0D6
:100360000197959A38D8959836D8482F492BC1F7D8
:1003700088EC90E040D88D9AEAE5F0E088EC90E0D7
:100380000197959A28D8959826D8482F492BC1F7D8
:10039000E1E0F0E0A9ECB0E07BE7E6DB8FEB11E019
:1003A000A1D7E2E7FDE187D7E1E0F0E0A0D78BD766
:1003B000A8EAB0E08C918F5F8C930091A80004367E
:1003C00010F009F001C001C05FC0E1E0F0E0ABEA6D
:1003D000B0E0DBDB8FE711E085D7ECE8FDE16BD720
:1003E000A6E1B4E0EBEAF0E048DB58D7EAE9FDE14A
:1003F00062D78FEB11E076D7A6E1B4E0E8ECF0E04D
:100400004BDB4CD7E4EAFDE156D7A298ABECB0E069
:100410009C9196FF04C09A9B0EC09F7B9C939A99D7
:100420000AC089E19F939927E6D79F919A9903C0C3
:1004300090649C9317C0A398ABECB0E09C9197FF9D
:1004400004C09B9B0EC09F779C939B990AC089E137
:100450009F939927D0D79F919B9903C090689C93B5
:100460000AC0A6CFA8ECB0E08C918F5F8C9380E09F
:100470008093A8009DCF8091C80081508093C800D0
:1004800080E08093A80094CF8D9AEAE5F0E088ECB4
:1004900090E00197959A9FD795989DD7482F492B23
:1004A000C1F788EC90E0A7D78D9AEAE5F0E088ECF8
:1004B00090E00197959A8FD795988DD7482F492B23
:1004C000C1F788EC90E097D7E0E0F0E0A8ECB0E06E
:1004D0007BE748DB8FEB11E005D7ECEBFDE1EBD6DA
:1004E000E1E0F0E004D781E08093A10084E0809314
:1004F000A20080E08093A80080E090E0ABEAB0E04A
:100500008D939C93E0D68CE043D7EED6E6EDFDE1EB
:10051000D2D6D7D6E0EFFDE1CED6E2E0F0E0E7D6E6
:1005200080EC806C87B967D8A5E7B0E08D939C9389
:1005300081EC806C87B95FD8A7E7B0E08D939C937E
:10054000E5E7F0E0D190E080FF240027BFD8ADE6DA
:10055000B0E0EDD8E7E7F0E0D190E080FF2400279D
:10056000B5D8A1E7B0E0E3D8E1E7F0E090D8EDE658
:10057000F0E088D892D9EDE0F0E046D8A9E7B0E005
:10058000EE0C000FE794DD92EC92E1E7F0E07FD80B
:10059000EDE6F0E077D872D9EDE0F0E035D8ABE7E2
:1005A000B0E0EE0C000FE794DD92EC92EBE7F0E0A8
:1005B000D190E0808FEFE7FE8827F82E082F86D8AD
:1005C000BBD82F933F934F935F93E9E7F0E0D1902F
:1005D000E0808FEFE7FE8827F82E082F77D85F910D
:1005E0004F913F912F91C3D8EDE0F0E0ADE7B0E03F
:1005F000A5DAEDE7F0E046D8ECEEFCE1A9D9B1D9F7
:1006000008F001C0C09AE0EFFCE1A2D9EDE7F0E00C
:1006100039D834D9EDE0F0E0A5E8B0E08FDAE0EFCA
:10062000FCE196D9EDE7F0E02DD837D9EDE0F0E028
:10063000A9E8B0E083DAE9E8F0E029D8E5E8F0E0FD
:1006400021D895D8EDE0F0E0A1E8B0E077DAE1E874
:10065000F0E011DBEDE0F0E0A1E9B0E06FDAE1E914
:10066000F0E015D8E4EFFCE16AD9D7D8EDE0F0E08E
:10067000ADE8B0E063DAE1E0F0E0A9ECB0E085DA03
:10068000E0E0F0E0A8ECB0E07EDAE0E0F0E0A0E14D
:10069000B0E079DA0F3F09F003C089E18093C80028
:1006A000E1E0F0E0A0E1B0E070DA0F3F5FEF1507A6
:1006B00009F006C08FEF90E0A9ECB0E08D939C9319
:1006C000E9ECF0E0D190E080FF240027FFD734D898
:1006D000E8EFFCE134D94BD8EDE0F0E0A8EBB0E076
:1006E0002DDAE8EBF0E0D3D7E8EBF0E0CBD795D804
:1006F000EDE0F0E0A8EBB0E021DAE8ECF0E0D0804B
:10070000EE24FF240027E2D717D8E8EBF0E0BAD7B1
:1007100084D8EDE0F0E0A8EBB0E010DAECEFFCE11B
:1007200017D9E8EBF0E0AED722D8EDE0F0E0A0EC8E
:10073000B0E004DAE0E0FDE10BD9E8EBF0E0A2D7AD
:1007400016D8EDE0F0E0A4ECB0E0F8D9E8EBF0E08A
:10075000ABDAEDE0F0E0ACEBB0E0F0D9E4E0FDE1E5
:10076000F7D8ECEBF0E08ED758D8EDE0F0E0ACEB4A
:10077000B0E0E4D9E8E0FDE1EBD8ECEBF0E082D7C3
:10078000F6D7EDE0F0E0A4EBB0E0D8D9E8E0FDE189
:10079000DFD8EDE6F0E076D740D8EDE0F0E0ADE66A
:1007A000B0E0CCD9ECE0FDE1D3D8EDE6F0E06AD7DB
:1007B000DED7EDE0F0E0ADE6B0E0C0D9E4EBF0E08C
:1007C00066D7EDE6F0E05ED728D8EDE0F0E0ADE6E4
:1007D000B0E0B4D9EDE6F0E05AD7EDE6F0E052D75C
:1007E0001CD8EDE0F0E0ADE6B0E0A8D9E0E1FDE135
:1007F000AFD8EDE6F0E046D7BAD7EDE0F0E0A5E9F6
:10080000B0E09CD9E8E0FDE1A3D8E1E7F0E03AD719
:1008100004D8EDE0F0E0A1E7B0E090D9ECE0FDE134
:1008200097D8E1E7F0E02ED7A2D7EDE0F0E0A1E71E
:10083000B0E084D9E4EBF0E02AD7E1E7F0E022D79A
:10084000ECD7EDE0F0E0A1E7B0E078D9E1E7F0E047
:100850001ED7E1E7F0E016D7E0D7EDE0F0E0A1E742
:10086000B0E06CD9E0E1FDE173D8E1E7F0E00AD750
:100870007ED7EDE0F0E0A9E9B0E060D9E9E9F0E089
:1008800006D7E5E9F0E0FED6F9D7EDE0F0E0ADE916
:10089000B0E054D9EDE9F0E0F5D6E4E1FDE158D857
:1008A00060D808F005C0ADE9B0E0E4E1FDE17AD838
:1008B000A5E7B0E00D911C91043B50E0150710F046
:1008C00009F001C054C0EDE7F0E0DCD6ECEEFCE14D
:1008D0003FD847D808F44BC0C098F5D48FE711E053
:1008E00001D5EAE0FEE1E7D48FEB19E0FBD4E4E2C6
:1008F000FEE1E1D4A6E1B4E0AF93BF93EDE7F0E011
:10090000C1D688D511E002E0BF91AF9160D8E6E191
:10091000F4E0A6E1B4E00DD9C1D481E08093A80051
:100920000091A8000A3010F009F017C08D9AE4E693
:10093000F0E086E990E00197959A4DD595984BD5D2
:10094000482F492BC1F782E390E055D5A8EAB0E0E3
:100950008C918F5F8C9308F4E3CFE2CDEDE7F0E06C
:1009600091D6ECEEFCE1F4D7FCD708F0B6CF8DEBD6
:1009700090EF90934D0080934C000027A3E3B0E0EC
:100980008C9182FB0EF401E040E0041709F027C0CF
:1009900088E290E030D5A2EAB0E08C918F5F8C9332
:1009A0008D9AEDE7F0E088EC90E00197959A13D5E9
:1009B000959811D5482F492BC1F785E08EBD89B791
:1009C000846089BF9A9BFECF0091A200063009F097
:1009D00003C081E08093A2008EB5887F8EBD009118
:1009E000A200013009F002C036D013C0023009F075
:1009F00002C0CCD00EC0033009F002C02CD109C017
:100A0000043009F002C0FAD104C0053009F001C079
:100A10008BD285EC806C87B9EED5A0E6B0E08D93E3
:100A20009C93A0E6B0E00D911C9142E050E01CD4F4
:100A3000A0E6B0E04D935C93A0E6B0E00D911C9170
:100A4000033250E0150710F009F001C002C0979A78
:100A500001C0979865CDA8EAB0E08C918F5F8C9328
:100A60000091A8000A3008F001C065C08FEB11E0CA
:100A700039D4EAE2FEE11FD4EDE7F0E003D6E4E189
:100A8000FDE166D76ED709F004C0E0E3FEE113D4C0
:100A900013C0A6E1B4E0AF93BF93EDE7F0E0F2D569
:100AA000B9D411E002E0BF91AF9191D7E6E1F4E053
:100AB000A6E1B4E03ED8F2D301E0F8D3E6E3FEE1EC
:100AC000FAD3EDE8F0E0DED5E8E1FDE141D749D722
:100AD00081E008F480E08F93EDE7F0E0D3D5E4E126
:100AE000FDE136D73ED781E009F080E09F91892B68
:100AF000882309F404C0ECE3FEE1DDD319C0E6E489
:100B0000FEE1D9D3A6E1B4E0AF93BF93EDE8F0E006
:100B1000B9D580D411E002E0BF91AF9158D7E6E19A
:100B2000F4E0A6E1B4E005D8B9D3E8E4FEE1C3D32C
:100B300080E08093A8008FE711E0D4D3EEE4FEE1DB
:100B4000BAD30091A100013009F004C0E4E6FEE14F
:100B5000B2D31BC0023009F004C0EAE6FEE1ABD319
:100B600014C0033009F004C0E0E7FEE1A4D30DC0D7
:100B7000043009F004C0E6E7FEE19DD306C005306D
:100B800009F003C0ECE7FEE196D30895AFEAB0E0C8
:100B9000EDE9F0E077D53ED48FEB11E0A3D3E2E8A6
:100BA000FEE189D3A8EAB0E08C918F5F8C9300912D
:100BB000A800053008F001C035C080E08093A8008F
:100BC000EDE9F0E05FD5E0E1FDE1C2D6CAD681E013
:100BD00008F080E08F93EDE9F0E054D5E4E0FDE12A
:100BE000B7D6BFD680E010F009F081E09F9189234D
:100BF000882309F40DC001E059D3EFEAF0E002E0E8
:100C0000A6E1B4E0A1D74AD3E6E9FEE154D30AC095
:100C1000EFEAF0E003E0A6E1B4E096D73FD3E6E9DF
:100C2000FEE149D38FE711E05DD3E4ECF0E02FD58E
:100C3000EDE9F0E027D59BD5EDE0F0E0E5D4A4EABE
:100C4000B0E0DD92EC9288E18093A90088E1809386
:100C5000AA00D2D10895A8EAB0E08C918F5F8C935E
:100C6000A5E7B0E00D911C9142E050E0FDD2ABEA67
:100C7000B0E04D935C93A7E7B0E00D911C9142E08A
:100C800050E0F2D2ADEAB0E04D935C930091A80041
:100C9000053008F001C087C08FE711E023D3EAE9EF
:100CA000FEE109D3ABEAB0E00D911C910A3050E0AF
:100CB000150708F009C002E0F9D2A6E1B4E0EBEABA
:100CC000F0E0DBD6EBD22AC0ABEAB0E00D911C918C
:100CD000093050E0150780E010F009F081E08F93B3
:100CE000ABEAB0E00D911C91043650E0150781E0AD
:100CF00008F080E09F918923882309F409C001E06E
:100D0000D5D2A6E1B4E0EBEAF0E0B7D6C7D206C090
:100D1000A6E1B4E0EBEAF0E0B0D6C0D28FEB11E090
:100D2000E1D2EEE9FEE1C7D2ADEAB0E00D911C914F
:100D30000A3050E0150708F009C002E0B7D2A6E17A
:100D4000B4E0EDEAF0E099D6A9D22AC0ADEAB0E06D
:100D50000D911C91093050E0150780E010F009F06A
:100D600081E08F93ADEAB0E00D911C91043650E024
:100D7000150781E008F080E09F918923882309F41A
:100D800009C001E093D2A6E1B4E0EDEAF0E075D647
:100D900085D206C0A6E1B4E0EDEAF0E06ED67ED2E0
:100DA00080E08093A8008FE717E09CD2ABEAB0E028
:100DB0000D911C914BE150E057D2A4EAB0E04D9365
:100DC0005C9382E18093A90082E18093AA0014D110
:100DD0008FEB17E087D2ADEAB0E00D911C914BE1AB
:100DE00050E042D2A4EAB0E04D935C9382E180935C
:100DF000A90082E18093AA00FFD00895AFEAB0E095
:100E0000EDE9F0E03FD406D3A8EAB0E08C918F5F23
:100E10008C930091A800053008F001C054C08FE702
:100E200011E060D2E2EAFEE146D2EDE9F0E02AD438
:100E3000E0E1FDE18DD595D581E008F080E08F936C
:100E4000EDE9F0E01FD4E4E0FDE182D58AD580E051
:100E500010F009F081E09F918923882309F40DC0E7
:100E600001E024D2EFEAF0E002E0A6E1B4E06CD6C3
:100E700015D2E8EAFEE11FD20AC0EFEAF0E003E093
:100E8000A6E1B4E061D60AD2E8EAFEE114D28FEB23
:100E900011E028D2E4E2FEE10ED2A6E1B4E0AF9385
:100EA000BF93EDE7F0E0EED3B5D211E002E0BF91E1
:100EB000AF918DD5E6E1F4E0A6E1B4E03AD6EED10B
:100EC00080E08093A8008FE719E00CD2E0ECF0E01E
:100ED000DED3EDE9F0E0D6D34AD4EDE0F0E094D3F0
:100EE000A4EAB0E0DD92EC9280E18093A90088E072
:100EF0008093AA0081D08FEB19E0F4D1ECEEFCE1F5
:100F000027D5EDE7F0E0BED388D4EDE0F0E07CD368
:100F1000A4EAB0E0DD92EC9280E18093A90088E041
:100F20008093AA0069D00895A8EAB0E08C918F5F01
:100F30008C9384EC806C87B95ED3A2E6B0E08D938D
:100F40009C93E2E6F0E0D190E080FF240027BED33E
:100F5000A4E6B0E0ECD3ECE1FDE1FAD4E4E6F0E0A5
:100F600091D35BD4EDE0F0E0A4E6B0E0E7D5E0E1BA
:100F7000FDE1EED4E4E6F0E085D3F9D3EDE0F0E076
:100F8000A4E6B0E0DBD5A8E6B0E0E4E6F0E07AD392
:100F900041D20091A8000A3008F001C02CC08FE7B0
:100FA00011E0A0D103E082D1EAEAFEE184D1A6E11A
:100FB000B4E0E0E6F0E061D571D182E0E3D1E8EBA6
:100FC000FEE179D104E072D18FEB11E08BD103E027
:100FD0006DD1EAEBFEE16FD1E8E6F0E004E0A6E1D6
:100FE000B4E0B2D55BD1E8ECFEE165D103E05ED1BF
:100FF00080E08093A800089581E08093A300A4EA94
:10100000B0E04D915C91A3EAB0E00D911127041777
:10101000150710F009F021C00091A300013009F07C
:1010200003C080E0AFD112C04091AA00041709F0BC
:1010300003C081E0A7D10AC04091A900041709F0BC
:1010400003C081E09FD102C084E09CD1A3EAB0E05C
:101050008C918F5F8C9308F4D2CFA4EAB0E00D910D
:101060001C9141E050E0040F151FA4EAB0E00D937D
:101070001C938091A4008093A3004091A90000914B
:10108000A300041710F009F021C00091A300013063
:1010900009F003C086E076D112C04091AA0004177F
:1010A00009F003C087E06ED10AC04091A90004177F
:1010B00009F003C087E066D102C083E063D1A3EAF0
:1010C000B0E08C918F5F8C9308F4D7CF08950F9286
:1010D0001F922F923F924F925F927F92AF92BF9258
:1010E0000F931F932F933F934F935F936F937F9330
:1010F0008F939F93AF93BF93CF93DF93EF93FF9320
:101100008FB78F93A1EAB0E08C918F5F8C93809121
:10111000A20081508093A2008D9AE4E6F0E088EC72
:1011200090E00197959A57D1959855D1482F492B22
:10113000C1F70091A100053010F009F001C003C013
:1011400081E08093A100BFD08FE711E0CBD0EAEC23
:10115000FEE1B1D08FEB11E0C5D00091A1000130CC
:1011600009F004C0E4EEFEE1A6D01BC0023009F095
:1011700004C0EEEFFEE19FD014C0033009F004C0BC
:10118000E8E1FFE198D00DC0043009F004C0E2E3CB
:10119000FFE191D006C0053009F003C0ECE4FFE1A7
:1011A0008AD0E1E0F0E0A3D00091A100013009F085
:1011B00003C083E088BB17C0023009F003C085E09C
:1011C00088BB11C0033009F003C089E088BB0BC0A5
:1011D000043009F003C081E188BB05C0053009F087
:1011E00002C081E288BB8F918FBFFF91EF91DF91A9
:1011F000CF91BF91AF919F918F917F916F915F91AF
:101200004F913F912F911F910F91BF90AF907F9081
:101210005F904F903F902F901F900F901895F894EB
:10122000FFCF00FC10D0089503D01ED001F8F9CFF5
:101230000024E89457FF02C009D0689400F80BD04E
:1012400010F80124089502D009D0089550954095D2
:101250004F5F5F4F0895E89417FF0895009510952C
:101260000F5F1F4F68940895352F242FE894452B66
:1012700011F468940895512F402F0027112780E121
:10128000440F551F001F111F021B130B416018F460
:10129000020F131F4E7F8A9599F70895A6E1B4E0D7
:1012A0008D91882311F06ED0FBCF089580E26AD033
:1012B0000A95E1F708953FD3802D11F063D0FBCF5D
:1012C000089580EC65C081E063D017D080E860C0ED
:1012D0008FE7213039F08FEB223021F08FE8233077
:1012E00009F08FEC810F54C080E852D0089588EE49
:1012F00093E081D03197D9F7089583E099277BC097
:101300008AEF90E078D0BF9A8E9A8C9ABE9A8B9A88
:101310008A9A929885E090E06ED09398C7989698B4
:10132000949AC69A939AEF93FF93E0E6F0E050D038
:10133000FF91EF9193985CD0939AEF93FF93E0E63F
:10134000F0E046D0FF91EF91939852D0939AEF93AB
:10135000FF93E0E6F0E03CD0FF91EF91939848D006
:10136000C698939AEF93FF93E0E6F0E031D0FF91B7
:10137000EF9193983DD088E20BD08EE009D086E0C3
:1013800007D00895929A829505D004D031D008955F
:101390009298F9CF859510F4C69A01C0C6988595A4
:1013A00010F4949A01C09498859510F4969A01C00F
:1013B0009698859510F4C79A01C0C798939AEF93B1
:1013C000FF93E0E6F0E004D0FF91EF919398089549
:1013D0003197F1F70895AE2FBF2F11974A2F4B2B5E
:1013E000E1F70895689462F80895E89462F8089522
:1013F00081E090E000C0EF93FF93EE27E82BE92B0C
:1014000031F0E8EEF3E03197F1F70197D1F7FF9172
:10141000EF9108958DE207FD8D938F2D881F802F0A
:10142000881F8F57082F6894F7F8802F87FF15C003
:1014300080958395082F80E38D938EE28D93802F86
:10144000815228F080E38D9399279C930895442737
:101450000A95802F09F192D01FC0805230F09EE48F
:101460009D9381E48D939D93EFCF4427DF92EF927C
:10147000FF920F938FE1801B11F0082F7FD085D052
:101480009EE29D930F91FF90EF90DF90442703958C
:10149000003209F4D7CF27D03F93ECE1F5E138E1F2
:1014A0002F2D1E2D0D2DFF24EE24DD244427000FAB
:1014B000111F221F88F42F923F923DD2102C3BD255
:1014C000202C39D2302C37D23197410DD21CE31C5D
:1014D000F01C3F902F9001C0339631963A9539F722
:1014E0003F9107D0B3CFDD0CEE1CFF1C0A95D9F756
:1014F0000895002719E058D08F93802B11F00395A1
:1015000001C08F911A95B9F7802F882309F49ACFDB
:101510008F91805D8D930A95D9F796CF0065CD1D8B
:1015200080B2E60E40597307A0ACB90350D6DC0177
:10153000286BEE0094357700CA9A3B0065CD1D00FC
:10154000B2E60E0059730700ACB90300D6DC010007
:101550006BEE0000357700009A3B0000CD1D0000C7
:10156000E60E000073070000B9030000DC01000074
:10157000EE000000770000003B000000F694E794C6
:10158000D79447950A95D1F7089500270DD08F93EA
:1015900003958F2D8E298D29842BC1F78F91805D26
:1015A0008D930A95D9F750CF1F930F93002710E220
:1015B000440FDD1CEE1CFF1C001F802F9AE0890BDE
:1015C00010F0082F43951A9599F7802F0F911F91CE
:1015D00008952093D0003093D1004093D2005093CF
:1015E000D30008952091D0003091D1004091D200D5
:1015F0005091D3000895369A3699FECF369A36998F
:10160000FECF84B195B108953DD0992711278F2D34
:10161000880F80E8F82A802F881F08F41FEF41F018
:101620008F57082F07FD04C0003240F08FEF01C034
:101630008827982FD82EE82EF82E09C08FE1801B1E
:10164000082FF694E794D79497950A95D1F711232C
:1016500051F09095D094E094F09481E0980F882711
:10166000D81EE81EF81E0F2DFE2CED2CD92E089545
:10167000D094E094F09491E0D90E9927E91EF91ED8
:1016800010950895D190E190F190019108952191E4
:101690003191419151910895102F90E8FF0C001F56
:1016A0000927990FF7941078652F90E8440F551F7C
:1016B0005927990F4795607800380895FF0C90E8F6
:1016C0009027110F9795F794092F0895102FBD2C8F
:1016D000DE2CEF2CF02E11234AF4B094D094E09439
:1016E000F0949FEFB91AD90AE90AF90A0EE1FF202E
:1016F00039F4FE2CED2CDB2CBB240850C2F76BC058
:1017000032F00A95BB0CDD1CEE1CFF1CF9CF01D09A
:10171000D5CFB7FE089590E8B91611F4D0FE08951C
:101720009FEFD91AE90AF90A09F403950895DD92A1
:10173000ED92FD920C930895502F2D2D3E2D4F2D9F
:10174000612F08952DEC3CEC4CEC5DE366270FC057
:1017500099DFF2DFDD24EE2490E8F92E0FE307C0D5
:1017600096DF05C02227332740E251E46627552340
:1017700051F1002381F190DF71F116270058505884
:101780000894050B18F407FD03C025C007FD23C00E
:10179000469537952795F694E794D79422D0FF2065
:1017A0002AF0DD0CEE1CFF1C015073F09D2D969568
:1017B00048F0DD203AF4EE202AF491E0D90E992782
:1017C000E91EF91E7BCF07C09FE7092FF92A9FEF7B
:1017D000D92EE92E0895DD24EE24FF2400271127B9
:1017E00008959F929924AA24BB2488E1D216E30687
:1017F000F40628F0D21AE30AF40A089401C0889487
:10180000991CAA1CBB1CDD0CEE1CFF1C8A9571F7F1
:10181000D92CEA2CFB2C9F9008953EDFE1F2503842
:10182000D1F21627005850580894051F12F418F4E6
:10183000CBCF08F0D0CF0AD0FF202AF0BB0CDD1CA4
:10184000EE1CFF1C3BCF0F5FFBF138CF9F9299241A
:10185000AA24BB24992788E1990CAA1CBB1CDD1C77
:10186000EE1CFF1C30F4920EA31EB41ED91EE91EFE
:10187000F91E8A9589F79F90089509DF0DDF50388A
:1018800029F090E869270CC00AF045D017CF5FE334
:1018900022273327442701C0FADEFEDE5038B1F399
:1018A000003899F3902F951B8BF312F434D0FACFB4
:1018B000983118F0222733274427983028F0232F17
:1018C000342F44279850F9CF992329F0469537951E
:1018D00027959A95D9F7912F962742F014D0B0F614
:1018E000F794E794D7940F5F8BF66ECF10D051F03A
:1018F00008F4BEDEFF2052F2DD0CEE1CFF1C01508E
:10190000CBF762CF68CFD20EE31EF41E0895D21A31
:10191000E30AF40A0895DF92EF92FF920F931F9368
:10192000D22EE32EF42E052F162F6F915F914F913B
:101930003F912F910895C895319600200895FBDFBF
:10194000D02CF9DFE02CF7DFF02CF5DF002D089527
:10195000F2DF202DF0DF302DEEDF402DECDF502DBB
:10196000089507FB00680EF40F7757FB50680EF4DC
:101970005F7707FD02C057FF05C0D216E306F406E5
:10198000050708952D153E054F05500708950024BD
:101990000D280E280F28002A0020089591E005C088
:1019A00092E003C094E001C098E0C5DF0D929A95E3
:1019B000E1F7089599278D9193958823E1F7939501
:1019C00011968C9311978E919A95D1F70895EA2FDD
:1019D000FB2F00244C918D9103948E32E1F711245A
:1019E0008D9113948823E1F71A94101640F41197FF
:1019F000202F2119239580E38D932A95E9F7113043
:101A000039F59927AE2FBF2FA00DB91FA00FB91F11
:101A10008C919C93853308F421C031E08E918E32F5
:101A2000E9F38D3241F0830F8A3319F480E331E01A
:101A300001C033278C93AE1789F7332341F0AE2FC3
:101A4000BF2FB8DF81E34D3209F4319680830895CA
:101A50008827E00DF81FE00FF81F80830895000F1E
:101A6000111F221F331F0895009510952095309562
:101A70000F5F1F4F2F4F3F4F0895019110810EC0F0
:101A800001911191219130810BC00191108117FFBB
:101A900005C03FEF2FEF04C0008111272227332715
:101AA00037FF03C0E1DF8DE28D93CF93DF93CF92B9
:101AB000DF92EF92AA24BB24CC24DD24EE2440E262
:101AC000CAE0DD2755E093E38881890F87FD9F7089
:101AD00083FD907F891B89935A95A9F7C0DFAA1CC3
:101AE000BB1CCC1CDD1CEE1C4A9551F7E894EFE0C2
:101AF000FF2782910ED0EB30E0F71EF068948A2D1C
:101B00000CD088278D93EF90DF90CF90DF91CF910D
:101B10000895982F829501D0892F8F70805D26F0CF
:101B2000803309F4089568948D93089588278D93E0
:101B3000089581918D938823E1F7089594E0819130
:101B40008D939A95E1F7089581918D930A9519F0F7
:101B50008823D1F70895EACFE199FECFEEBBFFBB12
:101B60003196089591E001C092E07B3751F47FB740
:101B7000F894F2DF8D918DBBE29AE19A9A95C9F7BC
:101B80007FBF7727089591E001C092E0E5DFE09AFA
:101B90008DB38D939A95D1F708951DCE73DD0023F3
:101BA000E2F3F5DE19F410DE0068089585E050D008
:101BB000FF0C001F04830FE70695F7946FD0506861
:101BC0006CDEB5DD139721E438E743ED5BEB25DEF2
:101BD00027E831ED43E15DE337D02EE03CE343EC11
:101BE0005DEB32D022E83DEA4BE25EE32DD02CEEF5
:101BF00032E846E75EEB28D020E931EE49EA5EE3C1
:101C000023D020E83FEE4FEF5EEB1ED024EC3FEFF9
:101C10004FE75FE319D08BDD139784818F5799F0DD
:101C20002AF4D82E0FEFE02EF02E04C0D82EEE248A
:101C3000FF2400274BDD28E132E741E35FE3EDDDE0
:101C400026DD34972ADE11C028DE21DD3497E5CD6C
:101C50000FB6F8944A925A92E42DF52DA42DB52D85
:101C6000480E8827581E0FBE08950FB6F894599055
:101C700049900FBE089506DD92DF29ED3BE54EED5C
:101C80005EE3CBCDFFDC802FFF0C001F901728F404
:101C9000091B881F0795F79408959DCD5FE340E8E1
:101CA00033272227089597CDEDDC0023E2F3D9F303
:101CB00088E0CEDF3CDD1196FF0C001F8FE7080F98
:101CC0000795F7940695F79483E08F9335DD2FDD24
:101CD0001397D8DC4CDDDBDC3897DFDD91E0D3DF18
:101CE0008F918A9511F08F93F1CFBFCF0000804084
:101CF0000000803F0000A0C10080FF430000804141
:101D00000000C041000020410000A04000007A44D3
:101D10000000C842000000000000704200409C40EB
:101D20002043414C49425241544520504F5745525F
:101D3000204D455445522020000020506C656173B1
:101D4000652072656C65617365206B65792E2E2E3A
:101D50002E200000446976005072657373206B6515
:101D60007920746F206D656D6F7279206469762EAD
:101D700000004469766973696F6E207361766564EB
:101D800020696E206D656D6F72790000496E707507
:101D90007420706F7765722F000020446976697334
:101DA000696F6E002057205B5345545D75702C5B46
:101DB0004D4F44455D646F776E2020003D3E504F8F
:101DC000574552205341564544212C5245535441C6
:101DD00052543D3E0000205357522D505752204D33
:101DE00065746572207665722E362E3031200000C3
:101DF00020202028522920594F3650495220323075
:101E0000313120202020202000004174656E74694B
:101E10006F6E2053575220544F204D555443482045
:101E2000212000005357523A0000205357523A00E5
:101E30002D2E2D2D00004C6F73733A00202D2E2D6A
:101E40002064422020002D00644220200000205306
:101E500057522F6442206D65746572202042616E76
:101E6000643A000038306D20000034306D200000EE
:101E700032306D20000031376D20000031306D2090
:101E800000005245414C2052462D504F574552209C
:101E90004F555420000020572000446972005265BD
:101EA00066005057523A0000570054656D702E433B
:101EB0006F6F6C65723A20004300506F7765722037
:101EC000537570706C793A005600202020204C6FBA
:101ED000772D506173732D46696C746572202020D4
:101EE000202000002053776974636820746F203EBF
:101EF0003E2042616E643A2038306D20000020534D
:101F0000776974636820746F203E3E2042616E647E
:101F10003A2034306D2000002053776974636820C4
:101F2000746F203E3E2042616E643A2032306D2054
:101F300000002053776974636820746F203E3E2050
:101F400042616E643A2031376D200000205377697A
:101F500074636820746F203E3E2042616E643A20B4
:061F600031306D2000008D
:00000001FF
